:020000040800F2
:1000000050050020E52500086D2500086F25000833
:100010007125000873250008752500080000000000
:10002000000000000000000000000000772500082C
:1000300079250008000000007B2500087D250008C8
:100040000126000805260008092600080D260008DC
:100050001126000815260008192600081D2600088C
:100060002126000825260008292600082D2600083C
:100070003126000835260008392600083D260008EC
:100080004126000845260008812500084926000869
:100090004D2600085126000855260008592600085C
:1000A0005D2600086126000865260008692600080C
:1000B0006D260008712600087526000879260008BC
:1000C0007D2600088126000885260008892600086C
:1000D0008D2600089126000895260008992600081C
:1000E0009D260008A1260008A5260008A9260008CC
:1000F000AD260008B1260008B5260008B92600087C
:10010000BD260008C1260008C5260008C92600082B
:10011000CD260008D1260008D5260008D9260008DB
:10012000DD260008E1260008E5260008E92600088B
:10013000ED260008F1260008F5260008F92600083B
:10014000FD260008012700080527000809270008E8
:100150000D27000811270008152700081927000897
:100160001D27000821270008252700082927000847
:100170002D2700083127000835270008000000005F
:10018000392700083D2700084127000845270008B7
:10019000492700084D270008512700085527000867
:1001A000592700085D2700086127000870B504463C
:1001B00000250CB9012070BD04F13C06706820B91F
:1001C000B5603070204600F075FA7068C10610D432
:1001D000706820F4885040F002007060204600F003
:1001E000C4F9B560716821F0020141F0010171604C
:1001F00000E0012500203070284670BD38B500F0C1
:1002000059F801D1022032BD00F05CF825D500F08C
:1002100032F846BF906820F00600002000F024F875
:100220000868426842F0806242F02002426000F0BA
:1002300035F806D1816811F0405F0ED100F00FF85B
:100240000BE0DFF81C14884202BFDFF818040268D4
:1002500012F0405F01D100F028F8002032BD816823
:1002600041F08041816070479060002414706FF00D
:100270002200186070475568DFF8EC03054045F42C
:10028000807555605868440505D5506820F40050C5
:1002900040F4805050605068C40470470868DFF82C
:1002A000CC130A6812F01F0F7047016841F08041BB
:1002B000016070470146002001F13C020090137874
:1002C000012B70470120107008688368DC0714D484
:1002D0008368DFF89C4343F001038360DFF89403F5
:1002E0000368B3FBF4F404EB4404009402E00098C8
:1002F000401E009000980028F9D10B689868C40748
:10030000704738B5044621680A684868920729D5BD
:10031000800627D5226CD00603D4226C42F40072EA
:100320002264886810F0405F04BFA069002812D1E1
:10033000C86A10F4700F02D0886842050BD4486870
:1003400020F020004860206C20F480702064206C35
:10035000C10400F066F8204600F07BFB21686FF0D6
:100360001200086021680A684868520730D5000604
:100370002ED5226CD00603D4226C42F400522264A3
:10038000886810F4401F1CD1886B10F4401F02D005
:100390008868420515D44868420512D4886810F070
:1003A000405F04BFA06900280BD1486820F080009E
:1003B0004860206C20F480502064206CC10500F05F
:1003C00030F8204600F028FC21686FF00C0008602F
:1003D000206802684168D2070FD549060DD500682C
:1003E000C1070AD5206C40F480302064204600F01C
:1003F00014FC21686FF00100086020680268416801
:1004000092060DD549010BD5626C42F0020262647E
:100410006FF020050560204600F000FC20680560B4
:1004200031BD03D4206C40F00100206470470068A7
:10043000C06C704778B502460020009092F83C30BE
:10044000012B01D1022072BD012082F83C0007245B
:100450000B6810680A2B11D30A3BC56803EB4303F2
:1004600000F077F8C460C3680D688C68A5F10A06CF
:1004700006EB4606B4402343C3600FE0056903EB77
:10048000430304FA03F325EA0303036103690D68D8
:100490008C6805EB4505AC40234303611F244B6882
:1004A000072B0CD25B1E456B00F051F84463436B85
:1004B0004D680C886E1E00F045F843631BE00D2B61
:1004C0000CD2DB1F056B00F042F80463036B4D6830
:1004D0000C88EE1F00F036F803630CE00D3BC56A94
:1004E00000F035F8C462C36A4D680C88A5F10D06AA
:1004F00000F028F8C3625A4B98421ED10C685B4842
:10050000122C03D1036843F4800303600B685A4C38
:10051000A34218BF112B10D1036843F400030360FA
:100520000868A04209D15349514C0B68B3FBF4F45D
:100530000A204443009400F010F8002182F83C1097
:10054000002072BD06EB8606B4402343704703EBE0
:1005500083039C4025EA0404704702E00098401E93
:10056000009000980028F9D17047404A116821F4A2
:1005700040311160136841680B431360026853688F
:1005800023F4807353605168036941EA0321516089
:10059000516821F040715160536881680B4353608A
:1005A000936823F4006393609368C1680B4393607E
:1005B0003249836A8B4210D0936823F07063936052
:1005C0009368816A0B439360936823F04053936070
:1005D0009368C16A0B43936007E0916821F07061F2
:1005E0009160916821F040519160916821F0020181
:1005F00091609168836941EA43019160016A002931
:1006000051680CD041F400615160516821F460419F
:1006100051605168436A5B1E41EA433101E021F4B5
:1006200000615160D16A21F47001D162D16AC3695D
:100630005B1E41EA0351D162916821F4007191601F
:100640009168036B41EA43219160916821F48061D4
:1006500091609168406941EA802191607047000093
:100660000020014008200140FEF9FFFF0423014063
:1006700040420F0078000020120000100100000F1F
:1006800081B00020009000224B48416841F4804135
:100690004160416801F48041009100990092036833
:1006A00043F080530360006800F080500090009891
:1006B00001B0704738B586B000F079F824683F4D36
:1006C000AC4228D10020009000223D48416941F40D
:1006D00000714161416901F400710091009900923B
:1006E0004021036843F0010303600322006800F027
:1006F000010000900098334801910292002103917B
:1007000001A900F0A9FA00220021122000F0B8FB94
:10071000122000F0D2FB07B030BD81B00068B0F10C
:10072000804F0BD1002124480091026842F0010261
:100730000260006800F001000090009801B070476E
:1007400081B00068204988420BD100221A480092EB
:10075000016841F004010160006800F004000090AD
:10076000009801B0704738B586B000F020F82468D2
:10077000154DAC4219D100200090022210480168AA
:1007800041F0080101604FF40051006800F00800DA
:10079000009000980D48019102920021039104916C
:1007A0000221059101A900F057FA07B030BD0446B7
:1007B00001A8142100F0ACBB4038024000210140E8
:1007C000303802400000024000080040000C0240A7
:1007D000F0B589B000F0A0FB00F0F0F801A81421FA
:1007E00000F096FB00200090DFF8B843DFF8B80374
:1007F000DFF8B8630168DFF8B85341F080010160A9
:10080000026802F0800200920022009900920368C0
:1008100043F001030360016801F0010100910099B8
:100820000092036843F008030360016801F00801C7
:100830000091009900924FF40051036843F0400387
:100840000360006800F0400000900098204600F02F
:10085000DFFA4FF40051019101220021039104912C
:10086000029201A9204600F0F7F96846102100F035
:100870004FFBD048D04C30604FF48031CF48B0624D
:1008800000220120F06170617160B2603261B2617A
:100890003262F262F26032633046FFF787FC062074
:1008A0000121009001910022029269463046FFF733
:1008B000C1FD00BFD6A01C2100F07AF800F028FB93
:1008C0000020606400214FF6FF70E064A1642165A0
:1008D000256404F1400000F064FB002100910191C7
:1008E00004F14000694600F039FD602100220291C8
:1008F00003920492069202A9042204F1400000F03F
:10090000A0FB04F14000FFF72EFF00BFBEA000F0E7
:100910004FF81C2100F0FCFA4FF08040606000218D
:10092000A1600020E0604FF0FF3160612161201D77
:1009300000F00CFB002100910191201D694600F0A0
:100940000DFD00210291002204910392069202A95A
:10095000201D00F053FB3046FFF750FC0021201D06
:1009600000F00AFB964E97489749984BC6E9060156
:1009700000229749C6E90823C6E90A214FF4967771
:10098000AF63042104F1400000F018FB2078002838
:10099000FCD196ED040B00F0A5F884ED200B51EC92
:1009A000100B00F001FDA863C82000F01BFDEDE76F
:1009B000D0E90023CDE9002302A8704780B592B0AA
:1009C00006A8302100F0A4FA01A8142100F0A0FA32
:1009D000002000904FF480337E48016841F0805140
:1009E00001600021006800F08050009000987A4873
:1009F0000091026822F4404242F4804202600122E7
:100A0000006800F44040009006A800990692022178
:100A10004FF480020C910D92042164220E910F92EA
:100A20000221042207931091119200F0EFFC0221A1
:100A30000291002203920F204FF4A05101900491E3
:100A40004FF480520592032101A800F05BFE13B021
:100A500000BD38B5554C5A4D2046FFF7E8FC2866D6
:100A600000F00EFF02460B4600205C4900F016FF26
:100A700000225B4B01F036F841EC100B01F0F3F86B
:100A800053EC102B5748584901F0F4F8574A584B8B
:100A900001F028F802460B460020564900F0FEFE01
:100AA000C5E90001D5E900234FF06630524901F055
:100AB00019F841EC100B85ED020B53EC102B0020C4
:100AC0004E4901F0D7F800224D4B00F0E7FE00221E
:100AD0004C4B01F007F8C5E904012046BDE832405F
:100AE000FFF78CBBF8B52DED068BB0EE408AF0EE2B
:100AF000608A01F091F9324C0546A06E6566281AAD
:100B000000F0BEFE41EC190BD4E90E0184ED0C9B04
:100B100053EC182B01F086F941EC180B84ED108B87
:100B200053EC182B51EC190B01F0A4F8D4E9122363
:100B300000F0D8FFD4E9162341EC1A0B84ED12AB78
:100B400051EC180B01F06EF953EC192B00F0A6FED6
:100B5000D4E9062341EC190B84ED149B84ED168B2C
:100B6000A56651EC180B01F085F8D4E90823064678
:100B70000F4651EC1A0B01F07DF832463B4600F06F
:100B8000B1FFD4E90A2305460E4651EC190B01F0DA
:100B900071F82A46334600F0A5FFBDEC068B41EC08
:100BA000100BF1BD0018024030380240080100204F
:100BB0000008004000210140800000200100000FDB
:100BC000000000209A9999999999B93F0000244012
:100BD00000003E4040380240007000400000B0403D
:100BE0000000F0BF3C9B1FEB60DB2D3F83DBB5DCDF
:100BF000E1796B3F0000F03F661271C000002240B7
:100C00000000144000004040000000000000000010
:100C1000000000000000000070477047704730B4CB
:100C2000002513E050F8042BD30744BFA9F10103BA
:100C30009A18091F042942F8045BFAD213468C075C
:100C400044BF15809B1CC90748BF1D7050F8041B8A
:100C50000029E7D130BC70472DE9F84702460B4622
:100C600000246D480F2101271D68A74007EA0508E9
:100C7000B84540F0C7805D68022D18BF122D4FEABD
:100C8000840911D1E50802EB850C09F01C05DCF89C
:100C900020E0D3F810A001FA05F62EEA06060AFABB
:100CA00005F53543CCF820504FEA440C032615686F
:100CB00006FA0CF66FEA060E1E7906F003060EEA37
:100CC000050506FA0CF6354315605D68012D18BF61
:100CD000022D03D0112D18BF122D10D19568DE689A
:100CE0000EEA050506FA0CF635439560556825EAC7
:100CF00007075D68C5F30015A5402F435760D76807
:100D00000EEA07059F6807FA0CF63543D5605D6863
:100D1000EF0077D50025009509F00C0907683F4ED4
:100D200047F48047076001FA09FE056805F480452D
:100D30000095009FA70856F8275025EA0E0E384D5B
:100D4000AA4208BF00252CD0364DAA4208BF012573
:100D500027D0354DAA4208BF022522D0334DAA42E2
:100D600008BF03251DD0324DAA4208BF042518D064
:100D7000304DAA4208BF052513D02F4DAA4208BF07
:100D800006250ED02D4DAA4208BF072509D02C4DAF
:100D9000AA4208BF082504D02A4DAA420CBF092543
:100DA0000A2505FA09F545EA0E0546F827506FEAC7
:100DB0000807254E356807EA050C5D68ED0348BF56
:100DC00048EA0C0CC6F800C0756807EA050C5D68B7
:100DD000AD0348BF48EA0C0CC6F804C0B56807EA82
:100DE000050C5D68ED0248BF48EA0C0CC6F808C067
:100DF000F56807EA050C5F68BD0248BF48EA0C0CBD
:100E0000C6F80CC0641C0F2C7FF62DAFBDE8F1872F
:100E100002B9090481617047443802400838014032
:100E2000000002400004024000080240000C0240A2
:100E3000001002400014024000180240001C024052
:100E40000020024000240240003C01400901020051
:100E500006D5294A00F00F00104400F8041C704722
:100E6000264B19547047264B19684FF6FF020002B3
:100E7000114000F4E06008432249084318607047BD
:100E800038B51F4B1C68C4F30223C3F10704052CBB
:100E900028BF04241D1D072D34BF0023DB1E0125A0
:100EA00005FA04F4641E2140994005FA03F35B1E21
:100EB0001A401143BDE83440C8E7012200F01F0189
:100EC000114BFFE78A40400943F82020704710B5D6
:100ED000401EB0F1807F01D3012010BD0B4C60603B
:100EE0000F214FF0FF30FFF7B1FF0021A160072075
:100EF0002060002010BD000018ED00E000E400E0DC
:100F00000CED00E00000FA0500E100E010E000E078
:100F1000002200F0F9BF000080B50B48016841F4E1
:100F200000710160026842F480620260016841F46D
:100F3000807101600320FFF796FF002000F0FEFFA4
:100F4000FFF79EFB002002BD003C024038B50400C4
:100F500001D1012032BD00F049F818B900F042F883
:100F6000FFF7DBFB02206870211D206800F0E7F826
:100F700001206870002032BD10B500F029F800F0A3
:100F80002CF81CBFDFF86C209042FFE703D1416CC6
:100F900041F400414164016841F001010160002019
:100FA00010BD38B5040001D1012032BD00F01EF89B
:100FB00018B900F017F8FFF7C3FBD3E710B500F03E
:100FC00007F800F00AF81CBFDFF828209042DDE7A0
:100FD00004460122206800F027B92068DFF81810C5
:100FE00088427047002129702046704704F1380577
:100FF00068787047000401400000014038B500F1F6
:1010000038042378012B01D1022032BD0123237043
:10101000022565704AB1042A0BD0082A0DD00C2A8B
:1010200004BF006800F05DF90AE0006800F006F90E
:1010300006E0006800F0CBF802E0006800F026F956
:1010400077E070B500F063F801D1022070BD00F0C8
:1010500065F832B1042A17D0082A28D00C2A39D0D2
:101060004AE03068294600F0E9F83068816941F0CB
:10107000080100F048F821F00401816131688A69B3
:10108000286902438A6137E03068294600F09FF8FA
:101090003068816941F4006100F035F821F4806125
:1010A00000F031F82A6941EA0221816124E03068C8
:1010B000294600F0EBF83068C16941F0080100F002
:1010C0001EF821F00401C1613168CA692869024330
:1010D000CA6111E03068294600F003F93068C1693F
:1010E00041F4006100F00BF821F4806100F007F892
:1010F0002A6941EA0221C16100F015F870BDC161A1
:101100003068C169704781613068816970470646FF
:1011100006F138040D462078012870470120207020
:101120000221617070470120607000212170002051
:1011300070470120607000212170002032BDF0B5A1
:10114000794C0568794B7A4E7A4FDFF8ECC1A042B2
:1011500018BFB0F1804F07D0604518BFB84203D028
:10116000B04218BF98420DD14A6825F0700515436A
:10117000A04218BFB0F1804F17D060451CBFB842E5
:10118000B04212D098421CBF6C4A90420DD06C4EB7
:10119000B0421CBF6B4A904207D06B4EB0421FBF9B
:1011A0006A4A90426A4EB04203D1CA6825F440753B
:1011B00015430560A0428D68C5620A68826212BF4D
:1011C00098420969016301224261F0BD000070B5D7
:1011D000026A554E22F010020262B042056A43686C
:1011E00084690A6824F4E64444EA02248A6825F003
:1011F000200545EA02151CBF4C4A90420DD1CA6831
:101200004E6925F0800545EA02158A6923F440639A
:10121000164325F0400543EA86034360846149682C
:101220008163056270BD000010B5036A01248C4023
:10123000A343036202FA01F1036A8BE0F0B5026A8C
:10124000520852000262066A446885690B688A681F
:1012500025F073051D4326F002061643324B9842D3
:101260001CBF324FB8420BD1CA684B6926F0080642
:1012700024F4407416438A691C4326F00406144380
:1012800044608561496841630662F0BD70B5026AD9
:1012900022F480720262056A4368C4690A688E6833
:1012A00024F07304144325F400751F4A45EA06250B
:1012B00090421CBF1D4EB0420DD1CA684E6925F444
:1012C000006545EA02258A6923F44053164325F454
:1012D000806543EA06134360C4614968C1630562DF
:1012E00070BD70B5026A104E22F480520262B042A4
:1012F000046A4268C3690D6823F4E64343EA0523A0
:101300008D6824F4005444EA05341CBF074DA842FC
:1013100004D14D6922F4804242EA85124260C361E1
:1013200049680164046270BD00000140000401408E
:10133000000C004000080040000400400040014054
:10134000004401400048014000180040001C0040DB
:10135000002000401943016210BD000030B500F1CB
:1013600038031A78012A01D1022030BD01221A70F7
:1013700002245C700268546824F0700454600468AD
:1013800065680A68154365600268946824F0800403
:10139000946002689468486804439460012159701D
:1013A0000020187030BD0000C1F30A5340F2FE3235
:1013B0009B1A14DDD3F120034FEAE17208DDC90264
:1013C00041EA505141F00040D840801850407047E9
:1013D00003F2E13010B1D24382F0004070470020A8
:1013E0007047000038B5044600F016FD14F1010FF7
:1013F000054602D004480178641800F00DFD401B3A
:10140000A042FAD331BD00BF6C0000202DE9F843A3
:10141000040017D02078B74EC10745D5B06800F05A
:101420000C00042807D0B06800F00C0008280BD18D
:101430007068410208D53068810335D5606800289E
:1014400040F0BA80012053E16068B0F5803F04D1DC
:10145000306840F48030306011E0B0F5A02F306883
:1014600006D140F480203060316841F4803105E0DD
:1014700020F480303060316821F480213160606870
:1014800068B100F0C9FC05463068810300F1948022
:1014900000F0C2FC401B6528F6D3032028E100F0D1
:1014A000BBFC05463068810340F1868000F0B4FC47
:1014B000401B6528F6D3F0E700F0AEFC401B022885
:1014C00040F2A780E9E7E06870B10121396000F0DF
:1014D000A3FC05463068810700F1CB8000F09CFC3E
:1014E000401B0228F6D9D8E7386000F095FC054685
:1014F0003168880763D500F08FFC401B0228F7D9BC
:10150000CBE7086000F088FC0546706F810775D551
:1015100000F082FC401B0228F7D9BEE70528306F97
:1015200006D140F004003067306F40F0010005E064
:10153000400840003067306F20F00400306741F20F
:101540008938A06868B100F067FC8146306F810778
:1015500000F19C8000F060FCA0EB09004045F5D351
:101560009BE700F059FC8146306F810740F18E8087
:1015700000F052FCA0EB09004045F5D38DE700F0E8
:101580004BFC401B022840F2968086E700F044FCAA
:10159000001B022840F2A7807FE70020386600F099
:1015A0003BFC04463068810140F1A18000F034FC2E
:1015B000001B0228F6D970E720784F4F81071BD512
:1015C000B06810F00C0F09D0B06800F00C000828CB
:1015D0007FF479AF706841023FF575AF30688107DD
:1015E00003D5E06801287FF42DAF3168206921F030
:1015F000F80141EAC0013160217808070DD5606922
:101600003E4900283FF47DAF01220A6000F004FC4F
:101610000546706F81077FF54FAF207841073AD5B7
:10162000306C0025C1000AD400950125316C41F0D1
:1016300080513164306C00F0805000900098DFF8E9
:10164000C080D8F80000C1051BD4D8F8000040F4D1
:101650008070C8F8000000F0DFFB8146D8F8000079
:10166000C1050ED400F0D8FBA0EB09000228F5D983
:1016700013E73068216920F0F80040EAC1003060CB
:10168000BAE7A06801287FF449AF4DE71DB1306C7F
:1016900020F080503064A06948B3B16801F00C01BB
:1016A00008293FF4CFAE02287FF477AF00203866D8
:1016B00000F0B2FB0546306881013FF560AFE2699A
:1016C000206A616A0243A06A400842EA8112401E11
:1016D00042EA0042E06A42EA006272600121396631
:1016E00000F09AFB0446306881017FF54FAF00207F
:1016F000BDE8F2830038024000004742800E4742B6
:10170000007000402DE9F04104000F4677D0404EB4
:10171000306800F00F00B84202D200F072F86ED1CB
:1017200020683C4D810712D5400703D5A96841F4D4
:10173000E051A9602078010703D5A86840F4604013
:10174000A860A968A06821F0F0010143A960217890
:10175000C8074CD56068012802D129688A0305E0D2
:10176000022818BF032803D129688A0103D446E060
:1017700029688A0743D5A968890840EA8100A860DA
:1017800000F04AFB8046A868616800F00C00B0EBEE
:10179000810F2CD000F040FBA0EB080041F2893112
:1017A0008842F0D3032020E02078410705D5AA68BD
:1017B000E06822F4E0520243AA602178080706D5C7
:1017C000A968206921F4604141EAC001A96000F0E4
:1017D00027F8AA681049114BC2F30312895CC8406C
:1017E0001860002000F0AAFB0020BDE8F0813068FE
:1017F00000F00F008742D7D200F003F8D4D00120C8
:10180000F3E73770316801F00F01B942704700000B
:10181000003C024000380240B82400087800002054
:1018200030B5144C606800F00C00042802D0082881
:1018300002D01DE0104830BD22682068002341021C
:1018400002F03F0204D525680B49C5F3881003E078
:1018500020680A49C0F38810A1FB000100F08EFB4C
:101860002168C1F30141491C4900B0FBF1F030BDD2
:10187000024830BD0438024000127A000024F4000F
:10188000014648B1B0FA80F18840C91CC1F58461B5
:10189000090501EBD021400570470000F0B540F28A
:1018A000FF7581EA030C0CF0004C15EA11541DBFC2
:1018B00015EA1357AC42AF42E5E0BC41C1F3130156
:1018C000C3F31303801A994143F4801304D2641EB6
:1018D0004000494180185941C90241EA5051B1FBC9
:1018E000F3F603FB1611A2FB0675D7EBC020A94146
:1018F00002D2761E80185941C90241EA5051B1FB0B
:10190000F3FE03FB1E11A2FB0E75D7EBC020A9410D
:1019100003D2AEF1010E80185941890241EA90517B
:10192000760546EA8E2EB1FBF3F603FB1611A2FBF9
:101930000675D7EB8020A94102D2761E8018594146
:10194000C90241EA50514EEA060EB1FBF3F603FB21
:101950001611A2FB0675D7EBC020A94102D2761E54
:1019600080185941C90241EA5051B1FBF3F703FB1A
:101970001711A2FB0735D3EBC020A94167F100077F
:101980000CBF004247F0010766F3D5274FEA1E312E
:10199000B80814F5806412DDBD0775F1004250EB04
:1019A0000E5051EB045111F5801F5CBF41EA0C0150
:1019B000F0BD4CF07F6141F0E0410020F0BDBD077B
:1019C0006D0840EA0E5041F48011D4F10104B4F1E5
:1019D00020060ADAC4F120060200E04001FA06F30C
:1019E000E1401843B24015430EE0342C13DCC6F13D
:1019F000200445EA40056D0820FA06F2154321FA55
:101A000006F0A1400D43002175F1004250F10000A5
:101A100051EB0C01F0BD00205FEA0C01F0BDCFB925
:101A200092185B41B3FA83F704BFB2FA82F6BF198A
:101A30000B3FB7F120062FBF02FA06F3BB40C7F1F8
:101A4000200622FA06F638BF3343BA401CB1E41927
:101A5000641E33E77F4231F00041B1FA81F404BFE4
:101A6000B0FA80F6A4190B3CB4F120062FBF00FA9F
:101A700006F1A140C4F1200620FA06F638BF314332
:101A8000A0403C1B1AE7AC421ABF05EA1357AF420D
:101A900012E050EA41061CBF52EA4306BFE750EA93
:101AA0004107304661461CBF41EA0551F0BD52EA8C
:101AB000430C08BFC143F0BD00204FF4001616EBE5
:101AC000410F98BF16EB430F08BF16EB410F24BF21
:101AD000C14305E016EB430F0CBF61464CEA0551CC
:101AE000F0BD000070B44FF0004591EA030F40F1E3
:101AF000A1816B40841A71EB030604D26E40001B77
:101B0000B141121973414FF4001C1CEB410F34BF5B
:101B10007CEB430683E00C0DA4EB1356362E00F34A
:101B20007C80012E45EAC32341DC43EA525312BFB5
:101B3000D20292025B08240545EAC12141EA5051D4
:101B4000D2EBC020994125D407D1B0FA80F610FA23
:101B500006F162D00020203608E0B1FA81F6B140EB
:101B6000C6F1200220FA02F21143B0404FEAF474A9
:101B7000B4EB465434F001064FEA74040AD8D6F5A3
:101B80000016760D04F00044F04061FA06F2504071
:101B9000F1404840C00A40EA415021F0004128BFCE
:101BA0005FEA500550F1000044EBD12135E0DB0A3B
:101BB00045EAC121C90AB6F120050EDD42EA02421A
:101BC000120CC5F1200603FA06F6EB4042EA0605C0
:101BD0006D42984161F100010DE062FA06F5F240B4
:101BE000554063FA06FC82EA0C02F3405A406D420B
:101BF000904161EB030111F4801F05D1641E620561
:101C000002D06D004041494121F48011430875F133
:101C1000004350F1000041EB045170BC70471CEBD5
:101C2000410F15D223F0004352EA43060BD04FEA8E
:101C30004C0CBCEB410F04D80C0D661E342EB7DDE6
:101C4000EBE7801A994150EA410608BF0021E4E71A
:101C500008BF1CEB430F28BF6FF00001DDE7000059
:101C600041EC100B01BD80B551EC100B00F096FB60
:101C7000F6E70000B0B581EA030C0CF0004C40F22E
:101C8000FF7515EA11541DBF15EA1357AC42AF4258
:101C900039E0E41923EA455343F48013C90241F0C3
:101CA000004141EA505EC7021100A7FB0202002872
:101CB0004FF00000EEFB01204FF00001E3FB072195
:101CC00018BF42F00102401800214941E3FB0E0118
:101CD000A4F580640F0302D252004041494154F1FF
:101CE00001046CDD470872F1004250F1000051EB35
:101CF0000451A1F580115CBF41EA0C01B0BD4CEA72
:101D000005510020B0BD05EA1357AC4214BFAF42E5
:101D100041E050EA410E1CBF52EA430E02E0614628
:101D20000020B0BD24423C441BD15FEA070EF6D030
:101D3000090302BF01460020AEF1140EB1FA81F78B
:101D4000AEEB070401FA07FE0C37C7F1200100FAD9
:101D500007F7C8404EEA000E23EA455343F48013C8
:101D6000A2E733F00043B3FA83F704BFB2FA82FE6E
:101D700077440B3FE41BB7F1200E2FBF02FA0EF39E
:101D8000BB40C7F1200E22FA0EFE38BF43EA0E0315
:101D9000BA40641C82E750EA410E14BF52EA430E77
:101DA0006FF000014FF4001717EB430F8ABF19467D
:101DB00017EB410FB5E74CEA05510020B0BDD4F157
:101DC0000104B4F120070FDAC4F12007520828BF3C
:101DD00042F0010210FA07F501FA07F7E1BF2A43C2
:101DE000E0403843E1400FE0352C98DCC7F1200497
:101DF00052EA400220FA07F218BF42F0010231FA1B
:101E000007F0A1400A43002172F1004250F10000A6
:101E100051EB0C01B0BD000001484068704700BFA5
:101E20006C00002070B44FF0004591EA030F7FF57D
:101E300061AE6B40841A71EB030603D2001BB14103
:101E4000121973414FF4001C1CEB410F34BF7CEBA3
:101E5000430442E00C0DA4EB1356352E4FDC45EA4B
:101E6000C323DB0A45EAC121C912B6F120050DDD05
:101E700063FA05F6EB4086EA0305124218BF45F007
:101E80000105C01851F100010CD213E062FA06F509
:101E9000F2405540F3415A40B340F3405A40801855
:101EA000594107D349085FEA30005FEA350528BF8A
:101EB00045F0010501F58011420875F1004250F12D
:101EC000000041EB04514E0016F5001F70BC38BFF6
:101ED00070470020090D090570471CEB410F10D217
:101EE00052EA43060BD0BCEB410F05D80C0DAB43B7
:101EF000661E342EB6DD02E0AB438018594170BC3B
:101F0000704770BC7047000000B500BF13009646D4
:101F10009446103928BFA0E80C50FAD85FEA417CFB
:101F200028BF0CC048BF40F8042BC90728BF20F8C1
:101F3000022B48BF00F8012B00BD000038B50D4D45
:101F40000D4B2A7804464FF47A711868B1FBF2F20F
:101F5000B0FBF2F0FEF7BBFF50B9102C08D2002204
:101F600021464FF0FF30FEF78BFFAC60002032BD02
:101F7000012032BD6C00002078000020D3BBD9B115
:101F8000B2F5803F5BD2022A1ED98C46B1FBF2F13A
:101F900002FB11C31B0443EA1043B3FBF2FC02FB38
:101FA0001C3380B240EA0343B3FBF2F002FB103271
:101FB00040EA0C4000237047022A05D98446B0FB52
:101FC000F2F002FB10C270474AB105D100F00102E5
:101FD00049085FEA3000704700220023704700F094
:101FE000DFB90B000200002100207047F7D3002268
:101FF00000237047904271EB030CF2D370B5B1FA35
:1020000081F4B3FA83F52C1BA340C4F1200532FA06
:1020100005F63343A2405FF00046E64002E05B086D
:102020005FEA3202841A71EB030524BF2046294679
:102030007641F4D302000B003000002170BD70B572
:10204000B1FA81F4B2FA82F5C4F120046419B4F152
:102050002006DAD3B2405FF00044F440002502E0ED
:1020600052085FEA3303C61A71EB020E24BF3046F2
:10207000714664416D41F3D302000B00200029003A
:1020800070BD00002DE9F84C2DED068B41EC180BCE
:1020900048004015401C82B014460DD14800401540
:1020A000401C01D1090303D151EC180BC80F30D1EA
:1020B00002B051EC180B25E153EC182B23F0004132
:1020C000B1F5801F22F000000BD20022002908BFCA
:1020D0000028009210D06A4651EC180B00F062F90B
:1020E00008E08A4E06EB1150009089498948034068
:1020F0001046194341EC180B51EC180B20F0000668
:1021000031F0004704BF002E834900F0FA80C80F69
:102110000AD0AFF3008002B04FF0FF30BDEC068B69
:102120006FF00041BDE8F48C51EC180B7B4A7C4BFE
:1021300000F070F90BD253EC182B00204FF08041C7
:10214000FFF798FD41EC180B0098401E009053ECEF
:10215000182B00207349FFF7C5FC41EC190B53EC19
:10216000182B00207049FFF7BDFC02460B4651ECCE
:10217000190BFFF793FB41EC180B53EC182BFFF7EF
:1021800079FD41EC1A0B53EC1A2B68486849FFF7AC
:1021900071FD684A684BFFF7A5FC53EC1A2BFFF75B
:1021A00069FD664A664BFFF79DFC53EC1A2BFFF75F
:1021B00061FD644A644BFFF795FC53EC1A2BFFF763
:1021C00059FD624A624BFFF78DFC53EC1A2BFFF767
:1021D00051FD604A604BFFF785FC53EC1A2BFFF76B
:1021E00049FD5E4A5E4BFFF77DFC53EC1A2BFFF76F
:1021F00041FD02460B4651EC190BFFF713FE53EC61
:10220000182BFFF737FD41EC180B009800F01AF976
:10221000002C41EC1A0B19D153EC1A2B514852499E
:10222000FFF728FD53EC182BFFF7FCFD53EC192B9F
:10223000FFF758FC04460D4653EC1A2B4FF0404074
:102240004A49FFF717FD22462B4658E053EC192B5D
:1022500034DD00204649FFF70DFD06460F4653ECDE
:10226000192B44484449FFF705FD04460D4653EC3D
:102270001A2B42484249FFF7FDFC82468B4653EC3D
:10228000182B40483A49FFF7F5FC02460B465046EA
:102290005946FFF7C7FD22462B46FFF723FC32467F
:1022A0003B46FFF71FFC04460D4653EC1A2B00205B
:1022B0003549FFF7DFFC22462B4620E04FF0C040B7
:1022C0003249FFF7D7FC06460F4653EC192B30482E
:1022D0003049FFF7CFFC04460D4653EC182B2E482F
:1022E0002A49FFF7C7FC02460B4620462946FFF75E
:1022F00099FD32463B46FFF7F5FB53EC1A2BFFF7EF
:10230000F1FB02B0BDEC068BBDE8F48C02FCFFFFD4
:102310000000E03FFFFF0F800000F0FFCD3B7F6635
:102320009EA0E63F0000F0BF0000F03FF7DE29BFAF
:10233000D8F8C23FF4B3FECC1A99C33F62CB68D938
:102340006F46C73FC6C912DAC471CC3F4AE98A94C6
:102350002449D23FF75F97999999D93FBC55555574
:102360005555E53F9EBC9AF71C7D7F3E422EE63FC9
:102370007BCBDB3FABA6320EE526553E7CC4BC7F53
:10238000DE27743E0EE526151344D33F4715F73F6D
:1023900044DF5DF80BAE543EFE822B65002271E6F1
:1023A0007047000010B5144600F002F8226010BD1E
:1023B000C1F30A5343B14A0012F5001F28D2A3F219
:1023C000FE32A1EB0251704750EA410C20D001F0DF
:1023D000004C31EA0C01B1FA81F204BFB0FA80F38B
:1023E000D2180B3AB2F120032CBF00FA03F191404E
:1023F00041EA0C013EBFC2F1200C20FA0CF3194354
:102400009040524240F2FD33D21A01EB0351704723
:10241000002270474FF4001C1CEB410F94BF1CEBD3
:10242000430F09E041EA030C50EA4C0C52EA0C0C51
:1024300003D2994208BF9042704714BF8B42824238
:1024400070470000C11768B14840401AB0FA80F2E6
:102450009040D21CC907C2F5846241EA025202EBE5
:10246000D0214005704700000E48016841F470011A
:10247000016000220C49086840F0010008608A6091
:102480000B680A480A4A03400B604A6000200B6848
:10249000084A23F480230B60C8604FF0006111608C
:1024A0007047000088ED00E000380240FFFFF6FEB4
:1024B0001030002408ED00E00000000000000000E3
:1024C000010203040607080930B501688468421850
:1024D000416802EB5103C9070BD54C4409E012F9DE
:1024E000011B12F8015B002904F8015B05D5491CAA
:1024F000F9D19A42F3D10C3030BD491EF1D5F8E73D
:1025000010B5074979441831064C7C44163404E070
:102510000A68081D114488470146A142F8D110BD40
:102520002C000000480000004EF68851CEF2000159
:10253000086840F470000860BFF34F8FBFF36F8FDF
:102540004FF00070E1EE100A70470000D3E6FFFF85
:10255000D000000080000020000000006DFFFFFFA1
:102560000402000028000000000000207047FEE781
:10257000FEE7FEE7FEE770477047704700F006B8D9
:102580000148FDF7BEBE0000080100200248416876
:1025900002788A18426070476C00002000F00DF845
:1025A000002801D0FFF7ACFFAFF300800020AFF3AD
:1025B0000080FEF70DF900F002F80120704700F0EE
:1025C00001B800000746384600F002F8FBE70000BB
:1025D00080B5AFF30080024A11001820ABBEFBE7C4
:1025E000260002000148804701480047692400088E
:1025F000F5250008AFF30080FFF796FFFFF7CEFF49
:10260000FFF7FEBFFFF7FEBFFFF7FEBFFFF7FEBFFE
:10261000FFF7FEBFFFF7FEBFFFF7FEBFFFF7FEBFEE
:10262000FFF7FEBFFFF7FEBFFFF7FEBFFFF7FEBFDE
:10263000FFF7FEBFFFF7FEBFFFF7FEBFFFF7FEBFCE
:10264000FFF7FEBFFFF7FEBFFFF7FEBFFFF7FEBFBE
:10265000FFF7FEBFFFF7FEBFFFF7FEBFFFF7FEBFAE
:10266000FFF7FEBFFFF7FEBFFFF7FEBFFFF7FEBF9E
:10267000FFF7FEBFFFF7FEBFFFF7FEBFFFF7FEBF8E
:10268000FFF7FEBFFFF7FEBFFFF7FEBFFFF7FEBF7E
:10269000FFF7FEBFFFF7FEBFFFF7FEBFFFF7FEBF6E
:1026A000FFF7FEBFFFF7FEBFFFF7FEBFFFF7FEBF5E
:1026B000FFF7FEBFFFF7FEBFFFF7FEBFFFF7FEBF4E
:1026C000FFF7FEBFFFF7FEBFFFF7FEBFFFF7FEBF3E
:1026D000FFF7FEBFFFF7FEBFFFF7FEBFFFF7FEBF2E
:1026E000FFF7FEBFFFF7FEBFFFF7FEBFFFF7FEBF1E
:1026F000FFF7FEBFFFF7FEBFFFF7FEBFFFF7FEBF0E
:10270000FFF7FEBFFFF7FEBFFFF7FEBFFFF7FEBFFD
:10271000FFF7FEBFFFF7FEBFFFF7FEBFFFF7FEBFED
:10272000FFF7FEBFFFF7FEBFFFF7FEBFFFF7FEBFDD
:10273000FFF7FEBFFFF7FEBFFFF7FEBFFFF7FEBFCD
:10274000FFF7FEBFFFF7FEBFFFF7FEBFFFF7FEBFBD
:10275000FFF7FEBFFFF7FEBFFFF7FEBFFFF7FEBFAD
:10276000FFF7FEBFC30002805140D4000001F90012
:082770000010FC000224F4003B
:04000005080025F5D5
:00000001FF
